:020000040000FA
:06000000F9EF20F01200F0
:020006001200E6
:080008000000000000000000F0
:0700100000000000000000E9
:0600180053EF1AF0120084
:02001E000300DD
:10002000100000000A0E0000070000000800000099
:10003000F80100000800000046420000CF01000067
:0400400017000000A5
:0C004400D9CFE6FFE1CFD9FF0B0EE1267B
:10005000DF6A010EDB6A040EF36E020EF3CFDBFFE4
:10006000010EF36E030EF3CFDBFF080EF36E040EEA
:10007000F3CFDBFF060EF36E050EF3CFDBFF010EB1
:10008000F36E060EF3CFDBFF010EF36E070EF3CF18
:10009000DBFF010EF36E080EF3CFDBFF090EDB6A08
:1000A0000A0EDB6AD398D38AD38C9B9CC26A300E2B
:1000B000C16E920EC06E0F010B0E5D6F5C6BC28045
:1000C000928092829286898A929AFB0E936E949085
:1000D000949294948C6A956A96909692030E8D12DF
:1000E000F80E8B148B6E8B802EEC0CF052EC0DF016
:1000F000010EF3C1DBFFD950010FE66E000EDA20CE
:10010000E66E89EC0DF0E552E552DF6ADFCF14F0C0
:10011000180EE76E1418E8AE02D0E73402D0E750AC
:10012000145C1BE2DFCFE9FFEA6AE9BEEA68D89017
:10013000E936EA36520EE926020EEA22EE68ED684A
:10014000DFCFE9FFEA6AE9BEEA68900EE926020E0F
:10015000EA22CD0EEF6EDF2AD9D7E668E668E668B8
:10016000E66AE66AE66AE66AE66A010EE66EE3ECCD
:1001700005F0146E090EE15E14500201BC6BF28EA4
:10018000F28C0B0EE15C02E2E16AE552E16EE552AF
:10019000E7CFD9FF1200D9CFE6FFE1CFD9FFE65272
:1001A000DF6AFD0EDBCFE9FFFE0EDBCFEAFFEECF0D
:1001B00008F0EDCF09F00850100B23E082A821D001
:1001C000100EE66EE66AB00EE66E100EE66EFEECFF
:1001D00008F0E552E552E552E552000902E002015D
:1001E000BC2BFD0EDBCFE9FFFE0EDBCFEAFFEE9866
:1001F000ED52FD0EDBCFE9FFFE0EDBCFEAFFEE8A0C
:10020000ED52FD0EDBCFE9FFFE0EDBCFEAFFEECFB6
:1002100008F0EDCF09F00850200B1BE082A819D0A0
:10022000200EE66EE66AB00EE66E100EE66EFEEC8E
:1002300008F0E552E552E552E552000902E00201FC
:10024000BC2BFD0EDBCFE9FFFE0EDBCFEAFFEE9A03
:10025000ED52FD0EDBCFE9FFFE0EDBCFEAFFEECF66
:1002600008F0EDCF09F00850400B23E082A821D020
:10027000400EE66EE66A500EE66E300EE66E20EC3C
:100280000AF0E552E552E552E552000902E00201AA
:10029000BC2BFD0EDBCFE9FFFE0EDBCFEAFFEE8EBF
:1002A000ED52FD0EDBCFE9FFFE0EDBCFEAFFEE9C49
:1002B000ED52FD0EDBCFE9FFFE0EDBCFEAFFEECF06
:1002C00008F0EDCF09F00850800B33E082A831D060
:1002D000800EE66EE66A500EE66E300EE66E20EC9C
:1002E0000AF0E552E552E552E552000902E002014A
:1002F000BC2B070E8B14DF6EF80E8B148B6EDFCFCA
:1003000014F0060EE76E1418E8AE02D0E73402D0FF
:10031000E750145C04E2DF508B10010F01D0010E96
:100320008B6EFD0EDBCFE9FFFE0EDBCFEAFFEE9E0C
:10033000ED6AE552E552E7CFD9FF1200D9CFE6FFCB
:10034000E1CFD9FF040EE126010EDE6EDE6ADE6A21
:10035000DD6ADD52DD52DECF14F0DECF15F0DECFE8
:1003600016F0DDCF17F0DD52DD52FE0EDB5008E057
:100370000001D8901436153616361736E804F9E120
:1003800014C0DFFF010E15C0DBFF020E16C0DBFF3D
:10039000030E17C0DBFFE66AE66AE66AE66AD9CFB3
:1003A000E9FFDACFEAFFEECFE6FFEECFE6FFEECFD2
:1003B000E6FFEFCFE6FF010EE66EE3EC05F0146E0C
:1003C000090EE15E1450040EE15C02E2E16AE552BE
:1003D000E16EE552E7CFD9FF1200D9CFE6FFE1CFBA
:1003E000D9FF040EE126010EDE6EDE6ADE6ADD6AEA
:1003F000DD52DD52DECF14F0DECF15F0DECF16F089
:10040000DDCF17F0DD52DD52FE0EDB5008E00001BB
:10041000D8901436153616361736E804F9E114C0AC
:10042000DFFF010E15C0DBFF020E16C0DBFF030E5F
:1004300017C0DBFFD9CFE9FFDACFEAFFEECFE6FF47
:10044000EECFE6FFEECFE6FFEFCFE6FFE66AE66A25
:10045000E66AE66A010EE66EB6DB146E090EE15E30
:100460001450040EE15C02E2E16AE552E16EE552ED
:10047000E7CFD9FF1200E6680F0EE66EE66AE66A7D
:10048000E66AE66AE66AE66AE66A9DDB146E090ECB
:10049000E15E14501200D9CFE6FFE1CFD9FF020E82
:1004A000E126FE0EEA6ADB34FE0BEA36E96E520EF6
:1004B000E926020EEA22EECFDEFFEDCFDDFF0E01D0
:1004C000105125E1DECF14F0DDCF15F0D890155096
:1004D00004E6030E145C000E155819E3DECF14F089
:1004E000DDCF15F0153411E21450F0080A0E155442
:1004F0000CE2DECF16F0DDCF17F0D890175004E6EF
:10050000100E165C0E0E175802E3010E106FFE0E51
:10051000EA6ADB34FE0BEA36E96E520EE926020E79
:10052000EA22EE68ED68DECF14F0DDCF15F014C0DE
:10053000F3FF15C0F4FF020EE15C02E2E16AE5524E
:10054000E16EE552E7CFD9FF1200D9CFE6FFE1CF48
:10055000D9FFE652FE0EDB50EA6A900FE96E020EFA
:10056000EA22EFCFDFFF0E010F5127E1DFCF14F0BA
:10057000D30EE76E1418E8AE02D0E73402D0E7508D
:10058000145C1BE3DFCF14F00A0EE76E1418E8AE1C
:1005900002D0143403D0E750D88014540CE2DFCFDB
:1005A00015F0320EE76E1518E8AE02D0E73402D02F
:1005B000E750155C02E3010E0F6FFE0EDB50EA6A96
:1005C000900FE96E020EEA22CD0EEF6EDFCF14F02F
:1005D000156A14BE156814C0F3FF15C0F4FFE55288
:1005E000E552E7CFD9FF1200D9CFE6FFE1CFD9FF1F
:1005F000FD0EDBCFE9FFFE0EDBCFEAFFEE6AED6A10
:10060000D80E0201E76EA819E8AE02D0E73402D096
:10061000E750A85D08E2FD0EDBCFE9FFFE0EDBCF61
:10062000EAFFEE80ED52D80EE76EA919E8AE02D0CF
:10063000E73402D0E750A95D08E2FD0EDBCFE9FF09
:10064000FE0EDBCFEAFFEE82ED52500EE76EA819E8
:10065000E8AE02D0A83503D0E750D880A85508E20C
:10066000FD0EDBCFE9FFFE0EDBCFEAFFEE84ED529D
:10067000500EE76EA919E8AE02D0A93503D0E750B5
:10068000D880A95508E2FD0EDBCFE9FFFE0EDBCFD7
:10069000EAFFEE86ED52AA5108E0FD0EDBCFE9FF3E
:1006A000FE0EDBCFEAFFEE88ED52AB5108E0FD0E07
:1006B000DBCFE9FFFE0EDBCFEAFFEE8AED52010150
:1006C000FA51FB1108E0FD0EDBCFE9FFFE0EDBCF98
:1006D000EAFFEE8CED52FA6BFB6B0201BC5108E0B5
:1006E000FD0EDBCFE9FFFE0EDBCFEAFFEE8EED5213
:1006F00080B408D0FD0EDBCFE9FFFE0EDBCFEAFFB2
:10070000EE52ED80FD0EDBCFE9FFFE0EDBCFEAFF00
:10071000020EE926000EEA22BCC2EFFFBC6BFD0E02
:10072000DBCFE9FFFE0EDBCFEAFF040EE926000E69
:10073000EA22F8C1EEFFF9C1EDFFE552E7CFD9FF9C
:100740001200D9CFE6FFE1CFD9FF020EE126DE6A23
:10075000DD6A830EC2140C09C26EC282C2B2FED719
:10076000C450176E166AC35000011624146E000E92
:100770001720156E14C0DEFFDD6ED9CFE9FFDACF8A
:10078000EAFFF40EEE5E010EED5AD9CFE9FFDACFA3
:10079000EAFF0A0E0D6E0E6AEECF08F0EDCF09F0FB
:1007A000E6EC1EF008C0EEFF09C0EDFFFD0EDBCF4A
:1007B000E9FFFE0EDBCFEAFF030EE926000EEA2278
:1007C000DFCFEFFF020EE15C02E2E16AE552E16E8B
:1007D000E552E7CFD9FF1200D9CFE6FFE1CFD9FF2D
:1007E000E652DF6A0101F86BF96B600EE66EACEC65
:1007F00020F0E552100EE66EE66A9A0EE66E1E0EC8
:10080000E66EFEEC08F0E552E552E552E552600E68
:10081000E66EACEC20F0E552200EE66EE66A9A0E2B
:10082000E66E1E0EE66EFEEC08F0E552E552E5526D
:10083000E552000903E00101F88F2BD0020EDF6EB4
:10084000DFCF14F0140EE76E1418E8AE02D0E734D0
:1008500002D0E750145C1DE2DFCFE9FFEA6AE9BE8F
:10086000EA682A0EE926020EEA22EF0402E10101FB
:10087000F881130EDF24E96EEA6AE9BEEA682A0EFF
:10088000E926020EEA22EF0402E10101F981DF2AE2
:10089000D7D7100EE66EE66A9D0EE66E1F0EE66E68
:1008A000FEEC08F0E552E552E552E552600EE66EC8
:1008B000ACEC20F0E552200EE66EE66A9D0EE66E88
:1008C0001F0EE66EFEEC08F0E552E552E552E552E9
:1008D000000903E00101F88F2BD0020EDF6EDFCF9D
:1008E00014F0140EE76E1418E8AE02D0E73402D00C
:1008F000E750145C1DE2DFCFE9FFEA6AE9BEEA686F
:100900002A0EE926020EEA22EF0402E10101F88331
:10091000130EDF24E96EEA6AE9BEEA682A0EE926C8
:10092000020EEA22EF0402E10101F983DF2AD7D7A0
:10093000100EE66EE66AB00EE66E100EE66EFEEC87
:1009400008F0E552E552E552E552600EE66EACEC79
:1009500020F0E552200EE66EE66AB00EE66E100E4E
:10096000E66EFEEC08F0E552E552E552E55200096C
:1009700002E00101F88F400EE66EE66A7A0EE66E3E
:100980003E0EE66E20EC0AF0E552E552E552E552E5
:10099000140EE66EACEC20F0E552800EE66EE66AD0
:1009A0007A0EE66E3E0EE66E20EC0AF0E552E55257
:1009B000E552E552000903E00101F88F35D0020E3F
:1009C000DF6EDFCF14F0060EE76E1418E8AE02D02B
:1009D000E73402D0E750145C1DE2DFCFE9FFEA6A9A
:1009E000E9BEEA68820EE926020EEA22EF0402E17D
:1009F0000101F885060EDF24E96EEA6AE9BEEA68BD
:100A0000820EE926020EEA22EF0402E10101F985D5
:100A1000DF2AD7D70201880502E10101F88502012A
:100A20008E0502E10101F985400EE66EE66A7D0E53
:100A3000E66E3F0EE66E20EC0AF0E552E552E55216
:100A4000E552140EE66EACEC20F0E552800EE66E38
:100A5000E66A7D0EE66E3F0EE66E20EC0AF0E55289
:100A6000E552E552E552000903E00101F88F35D067
:100A7000020EDF6EDFCF14F0060EE76E1418E8AE3C
:100A800002D0E73402D0E750145C1DE2DFCFE9FF6B
:100A9000EA6AE9BEEA68820EE926020EEA22EF045B
:100AA00002E10101F887060EDF24E96EEA6AE9BE79
:100AB000EA68820EE926020EEA22EF0402E1010151
:100AC000F987DF2AD7D70201880502E10101F887FB
:100AD00002018E0502E10101F987400EE66EE66A29
:100AE000500EE66E300EE66E20EC0AF0E552E5524E
:100AF000E552E552140EE66EACEC20F0E552800EA5
:100B0000E66EE66A500EE66E300EE66E20EC0AF0F7
:100B1000E552E552E552E552000902E00101F88F85
:100B2000100EE66EE66AD6DAE552E5526E0EE66E15
:100B3000ACEC20F0E552200EE66EE66ACBDAE55228
:100B4000E552000903E00101F88F34D00201D8908A
:100B5000B55104E6340EB45D080EB55902E2010148
:100B6000F8890201B53507E2B45154080B0EB555AA
:100B700002E20101F88B0201B85102E00101F88D97
:100B80000201D890B75104E6340EB65D080EB7598D
:100B900002E20101F9890201B73507E2B6515408B2
:100BA0000B0EB75502E20101F98B0201B95102E0C7
:100BB0000101F98DF8C1F3FFF9C1F4FFE552E552E7
:100BC000E7CFD9FF1200D9CFE6FFE1CFD9FF180E4A
:100BD000E126140EDB6A150EDB6A160EDB6A170EB1
:100BE000DB6AD950FA0FE96EFF0EDA20EA6E0101D6
:100BF000FC51EE10FC6FFD51EE10FD6FFE51EE103A
:100C0000FE6FFF51EE10FF6FF60EDBCF14F0F70E04
:100C1000DBCF15F0F80EDBCF16F0F90EDBCF17F0B7
:100C2000141E151E161E171EFC0EE96E010EEA6E2E
:100C3000EE501414FC6FEE501514FD6FEE501614A8
:100C4000FE6FEE501714FF6F140EFCC1DBFF150E84
:100C5000FDC1DBFF160EFEC1DBFF170EFFC1DBFF80
:100C6000140EDBCF14F0150EDBCF15F0160EDBCF14
:100C700016F0170EDBCF17F01450E76E020EE7CF19
:100C8000DBFF140EDBCF14F0150EDBCF15F0160EC4
:100C9000DBCF16F0170EDBCF17F0080ED890173207
:100CA000163215321432E806F9E1140E14C0DBFFD7
:100CB000150E15C0DBFF160E16C0DBFF170E17C092
:100CC000DBFF0F0E146E156A166A176AD950140FDF
:100CD000E96EDACFEAFFEE501416EE501516EE501C
:100CE0001616EE501716030E14C0DBFF140EDBCFE2
:100CF00014F0150EDBCF15F0160EDBCF16F0170E25
:100D0000DBCF17F0040ED89017321632153214329A
:100D1000E806F9E1140E14C0DBFF150E15C0DBFF69
:100D2000160E16C0DBFF170E17C0DBFF140EDBCF4D
:100D300014F0150EDBCF15F0160EDBCF16F0170EE4
:100D4000DBCF17F01450DF6E140EDBCF14F0150E4E
:100D5000DBCF15F0160EDBCF16F0170EDBCF17F03A
:100D6000080ED8901732163215321432E806F9E11F
:100D7000140E14C0DBFF150E15C0DBFF160E16C0D7
:100D8000DBFF170E17C0DBFF0F0E146E156A166A15
:100D9000176AD950140FE96EDACFEAFFEE50141635
:100DA000EE501516EE501616EE501716010E14C022
:100DB000DBFFFE0EDB50100FE76E060EE7CFDBFF0A
:100DC000070EDFCFDBFF010EDB50E76E080EE7CF2B
:100DD000DBFF090EDB6A770EF36E0A0EF3CFDBFF43
:100DE000AA0EF36E0B0EF3CFDBFF060EE66ED950A4
:100DF000060FE66E000EDA20E66E7AEC0BF0E55296
:100E0000E552E552E76E0C0EE7CFDBFFFE0EDB503E
:100E1000100FE76E0D0EE7CFDBFF020EDB50E76E23
:100E20000E0EE7CFDBFF030EDB50E76E0F0EE7CFB2
:100E3000DBFF100EDB6A770EF36E110EF3CFDBFFD4
:100E4000AA0EF36E120EF3CFDBFF060EE66ED9503C
:100E50000D0FE66E000EDA20E66E7AEC0BF0E5522E
:100E6000E552E552E76E130EE7CFDBFFD950040FD2
:100E7000E66E000EDA20E66E100EE66EC70EE66E27
:100E8000010EE66E08EC0DF0146E050EE15E1450D6
:100E9000180EE15C02E2E16AE552E16EE552E7CF4D
:100EA000D9FF1200D9CFE6FFE1CFD9FFE652DF6AC2
:100EB000000EE66E020EE66E100EE66ECE0EE66ECA
:100EC000020EE66E08EC0DF0146E050EE15E145095
:100ED000060EE66E020EE66E020EE66E7AEC0BF081
:100EE000E552E552E5520201085D0EE1060EE66E9E
:100EF000090EE66E020EE66E7AEC0BF0E552E55254
:100F0000E55202010F5D02E0DF6ADED0070E09152F
:100F1000116F070E0215106F0951E840E840E840D4
:100F20001F0B010B136F0251E840E840E8401F0B14
:100F3000010B126F09390F0B010B156F02390F0BE3
:100F4000010B146F0951E00BE838E840030B176FF1
:100F50000251E00BE838E840030B166F0945010B1E
:100F6000010B196F0245010B010B186F0F0E0B15CA
:100F70001C6F1D6B156E146A0A5114241C6F000E31
:100F800015201D6F0F0E04151A6F1B6B156E146A5A
:100F9000035114241A6F000E15201B6F0C51206F83
:100FA000216B0CC214F021C215F0040ED890143637
:100FB0001536E804FBE102010B390F0B1424206FF6
:100FC000000E1520216F05511E6F1F6B05C214F016
:100FD0001FC215F0040ED89014361536E804FBE154
:100FE000020104390F0B14241E6F000E15201F6F11
:100FF0001F0E0D5D246F256B040E000A06E0020132
:10100000D89024372537E804FBE124C214F025C228
:1010100015F0D89015321432020124511424246F93
:1010200025511520256F1F0E065D226F236B040EC0
:10103000000A06E00201D89022372337E804FBE1DA
:1010400022C214F023C215F0D890153214320201D6
:1010500022511424226F23511520236F200E0E5D80
:10106000286F296B040E000A06E00201D890283789
:101070002937E804FBE128C214F029C215F0D89002
:1010800015321432020128511424286F29511520D9
:10109000296F200E075D266F276B040E000A06E0FD
:1010A0000201D89026372737E804FBE126C214F066
:1010B00027C215F0D890153214320201265114249B
:1010C000266F27511520276FDF50E552E552E7CFF5
:1010D000D9FF1200D9CFE6FFE1CFD9FFE652DF6A90
:1010E000D950FD0FE96EFF0EDA20EA6E100EEE18F1
:1010F0000AE1ED5008E1790EE66E520EE66EF3EC71
:101100000CF0E552E552D950FD0FE96EFF0EDA20E2
:10111000EA6E200EEE186CE1ED506AE182A868D00C
:10112000898AAC0EE66E020EE66E080EE66E6B0E57
:10113000E66E540EE66E08EC0DF0146E050EE15EE0
:101140001450020EE66EAE0EE66E020EE66ED2DAB7
:10115000E552E552E5520201B05D0DE1020EE66E88
:10116000B10EE66E020EE66EC5DAE552E552E552C4
:101170000201B35D02E0DF6A3BD0AFC2E6FFAEC260
:10118000E6FF73DBE552E552F3CFB4F2F4CFB5F2EC
:10119000B2C2E6FFB1C2E6FF68DBE552E552F3CF2B
:1011A000B6F2F4CFB7F20201AF51E00BE838E840F5
:1011B000010BB86FB251E00BE838E840010BB96F92
:1011C000060EAFC2E7FF070B04E0E742E79EE80622
:1011D000FCE1E7500201BA6F060EB2C2E7FF070B4F
:1011E00004E0E742E79EE806FCE1E7500201BB6F3E
:1011F000DF50E552E552E7CFD9FF1200D9CFE6FF25
:10120000E1CFD9FF030EE126020EDB6AD950FB0FB6
:10121000E96EFF0EDA20EA6E100EEE181AE1ED50BC
:1012200018E1E668E668E668E66AE66AE66AE66A9B
:10123000E66A010EE66EC7DC146E090EE15E14501C
:10124000FD0EDBCFE6FFFE0EDBCFE6FFCCDBE5528B
:10125000E552D950FB0FE96EFF0EDA20EA6E200E40
:10126000EE1801E0DFD0ED5001E0DCD082A8DAD04A
:10127000898ACFC114F0D0C115F0D1C116F0D2C106
:1012800017F0141E151E161E171E14C0E6FF15C0FB
:10129000E6FF16C0E6FF17C0E6FFCFC1E6FFD0C1EC
:1012A000E6FFD1C1E6FFD2C1E6FF010EE66E8BDCA0
:1012B000186E090EE15E18502A0EE66E020EE66EFA
:1012C000280EE66EDC0EE66E040EE66EA1DB146EF2
:1012D000050EE15E1450120EE66E2C0EE66E020E46
:1012E000E66E08DAE552E552E55202013E5D0DE197
:1012F000120EE66E3F0EE66E020EE66EFBD9E5526A
:10130000E552E5520201515D03E0020EDB6A8AD02C
:10131000DF6ADFCF14F0180EE76E1418E8AE02D0C3
:10132000E73402D0E750145C01E37CD0DF407F0B50
:10133000DF24E76E010EE7CFDBFFDFCF14F00B0EEB
:10134000E76E1418E8AE02D0143403D0E750D8800A
:10135000145402E2010EDB2A010EDB50030FE96E8A
:10136000EA6AE9BEEA682A0EE926020EEA22EF508E
:10137000E66E010EDB50020FE96EEA6AE9BEEA682A
:101380002A0EE926020EEA22EF50E66E6EDAE552E8
:10139000E552F3CF14F0F4CF15F0DFCFE9FFEA6A9E
:1013A000E9BEEA68D890E936EA36520EE926020E1E
:1013B000EA2214C0EEFF15C0EDFF010EDB50040F52
:1013C000E96EEA6AE9BEEA682A0EE926020EEA2216
:1013D000EF50E66E010EDB50030FE96EEA6AE9BEDC
:1013E000EA682A0EE926020EEA22EF50E66E9BDA40
:1013F000E552E552F3CF14F0F4CF15F0DF28E96E93
:10140000EA6AE9BEEA68D890E936EA36520EE92679
:10141000020EEA2214C0EEFF15C0EDFF020EDF241B
:10142000DF6E77D7020EDB50146E030EE15C02E232
:10143000E16AE552E16E1450E552E7CFD9FF1200A0
:10144000D9CFE6FFE1CFD9FF070EE126040EDB6A14
:10145000050EDB6A060EDB6AD950FB0FE96EFF0E44
:10146000DA20EA6E400EEE180BE1ED5009E1FD0EB8
:10147000DBCFE6FFFE0EDBCFE6FFB5DAE552E55245
:10148000D950FB0FE96EFF0EDA20EA6E800EEE18DF
:1014900001E022D1ED5001E01FD182A81DD1898A3F
:1014A000820EE66E020EE66E0E0EE66EEA0EE66E38
:1014B0000E0EE66EADDA146E050EE15E1450050EEA
:1014C000E66E840EE66E020EE66E14D9E552E55223
:1014D000E5520201895D0DE1050EE66E8A0EE66EAB
:1014E000020EE66E07D9E552E552E55202018F5D24
:1014F00003E0060EDB6AF0D0DE52020EDD6E070E50
:101500008B14E76E040EE7CFDBFFDB06DBCFE6FFD5
:10151000050EE552D880E754E76E050EE7CFDBFFF6
:10152000DF6ADFCF14F0180EE76E1418E8AE02D0B1
:10153000E73402D0E750145C01E3C5D0010EDB288C
:10154000E96EEA6AE9BEEA68820EE926020EEA223C
:10155000EF50E66E010EDBCFE9FFEA6AE9BEEA680A
:10156000820EE926020EEA22EF50E66E7ED9E5529F
:10157000E552020EF3CFDBFF030EF4CFDBFF020ECA
:10158000DBCFE6FF030EDBCFE6FF3BEC20F0E552BE
:10159000E552E66E040EDB50E824DF24EA6A900F81
:1015A000E96E020EEA22E552E750EF6E010EDB2AE9
:1015B000DB28E96EEA6AE9BEEA68820EE926020ED5
:1015C000EA22EF50E66E010EDBCFE9FFEA6AE9BEE0
:1015D000EA68820EE926020EEA22EF50E66EA3D9EF
:1015E000E552E552020EF3CFDBFF030EF4CFDBFF33
:1015F000020EDBCFE6FF030EDBCFE6FF3BEC20F075
:10160000E552E552E66E050EDB50E824DF24010FBB
:10161000EA6A900FE96E020EEA22E552E750EF6E99
:10162000010EDB50020FE76E010EE7CFDBFFDB2878
:10163000E96EEA6AE9BEEA68820EE926020EEA224B
:10164000EF50E66E010EDBCFE9FFEA6AE9BEEA6819
:10165000820EE926020EEA22EF50E66E06D9E55226
:10166000E552020EF3CFDBFF030EF4CFDBFF020ED9
:10167000DBCF15F0030EDBCF16F0D8901632153203
:10168000E804FBE1110E155E010E165A0C0E146EE5
:101690000E6EDFCF09F0CCEC1EF009C0E9FFEA6A5C
:1016A000E9BEEA68A80EE926020EEA2215C0EFFF9D
:1016B000010EDB50030FE76E010EE7CFDBFF0C0ED0
:1016C000DF24DF6E2ED7020188390F0B010BAA6FC2
:1016D0008E390F0B010BAB6F060EDB50146E070E2D
:1016E000E15C02E2E16AE552E16E1450E552E7CFB7
:1016F000D9FF1200D9CFE6FFE1CFD9FF070EE126CF
:10170000410EF36E020EF3CFDBFF030EDB6A040E15
:10171000DB6A050EDB6A060EDB6ADF6AFC0EDB5055
:10172000DF5C01E38DD0010EDB6ADBCF14F0080E25
:10173000E76E1418E8AE02D0E73402D0E750145C2C
:1017400001E37CD0800E156E010EDB5015C0E7FF63
:10175000070B04E0E742E79EE806FCE1E750146E61
:10176000DF50E76EFD0EDBCFE9FFFE0EDBCFEAFFB9
:10177000E750E926000EEA22EF501414E76E030E3C
:10178000E7CFDBFF010EDBCFE6FF070EE552D88087
:10179000E754146E030EDB5014C0E7FFE75204E079
:1017A000E8427F0BE706FCE1E76E030EE7CFDBFFC5
:1017B000DBCFE6FF020EDB50800BE844010BE55265
:1017C000E718E76E040EE7CFDBFFDBCFE6FF020E84
:1017D000DB50010BE552E718E76E050EE7CFDBFFA4
:1017E000040EDBCFE6FF020EDB50020BE8407F0B5E
:1017F000E552E718E76E060EE7CFDBFF020EDB507F
:10180000020D020EF3CFDBFF040EDBCFE6FF050E69
:10181000DB50E824156E060EDB50040DF350151056
:10182000E552E710146E020EDB50F80B1410E76E51
:10183000020EE7CFDBFF010EDB2A77D7DF2A6ED758
:10184000020EDB50146E070EE15C02E2E16AE55223
:10185000E16E1450E552E7CFD9FF12009496949AA6
:10186000320EC66EC79C9E961200D9CFE6FFE1CF1E
:10187000D9FF020EE126DE6ADD6AFD0EDB500F0B9A
:10188000DE6EDD6ADECF16F0DDCF17F016C017F082
:10189000166AFE0EDB501624146E000E172014C0BC
:1018A000DEFFDD6EDECF14F0DDCF15F0000E145E2E
:1018B000020E155A14C0DEFF15C0DDFFDECF14F096
:1018C000DDCF15F0800E151408E1DECF16F0DDCF68
:1018D00017F0D890173216320BD0DECF16F0DDCFCE
:1018E00017F0D89017321632000E1626800E1722E7
:1018F000DE501624146EDD501720156E14C0DEFF66
:10190000DD6EDECF14F0DDCF15F014C0F3FF15C08F
:10191000F4FF020EE15C02E2E16AE552E16EE5529B
:10192000E7CFD9FF1200D9CFE6FFE1CFD9FF020EF2
:10193000E126DE6ADD6AFD0EDB50DE6EDD6ADECF9B
:1019400016F0DDCF17F0040ED89016361736E804DF
:10195000FBE1FE0EDB380F0B1624146E000E172071
:1019600014C0DEFFDD6EDECF14F0DDCF15F0000E0B
:10197000145E020E155A14C0DEFF15C0DDFFDECF67
:1019800014F0DDCF15F0800E151408E1DECF16F04F
:10199000DDCF17F0D890173216320BD0DECF16F00D
:1019A000DDCF17F0D89017321632000E1626800EB3
:1019B0001722DE501624146EDD50172014C0DEFFEF
:1019C000DD6EDECF14F0DDCF15F014C0F3FF15C0CF
:1019D000F4FF020EE15C02E2E16AE552E16EE552DB
:1019E000E7CFD9FF1200D9CFE6FFE1CFD9FF899A1F
:1019F000FE0EDB50C96E9EA6FED79E96FD0EDB50F6
:101A0000C96E9EA6FED79E96E552E7CFD9FF12007B
:101A1000D9CFE6FFE1CFD9FFE652FA0EDBCFE9FFDF
:101A2000FB0EDBCFEAFFFE0EDBCFEFFF010EE76E12
:101A3000FA0EDBCFE9FFFB0EDBCFEAFFE750E9262A
:101A4000000EEA22FD0EDBCFEFFF899ADF6AFC0E63
:101A5000DB50DF5C21E2DF50E76EFA0EDBCFE9FFFF
:101A6000FB0EDBCFEAFFE750E926000EEA22EF503B
:101A7000C96E9EA6FED79E96DF50E76EFA0EDBCFAC
:101A8000E9FFFB0EDBCFEAFFE750E926000EEA2272
:101A9000C9CFEFFFDF2ADBD7898AE552E552E7CFCE
:101AA000D9FF1200CD88CD8A9F909D809E90CD82D7
:101AB000CD8012000101FA8D1200D9CFE6FFE1CFEF
:101AC000D9FF020EE126DE6ADD6A830EC214000928
:101AD000C26EC282C2B2FED7C450176E166AC3501D
:101AE0001624146E000E172014C0DEFFDD6EDECF4C
:101AF00014F0DDCF15F014C0F3FF15C0F4FF020E93
:101B0000E15C02E2E16AE552E16EE552E7CFD9FF1E
:021B10001200C1
:0E1B1200D9CFE6FFE1CFD9FF800EE66E7CEC66
:101B200018F0E552729E728CFD0EDBCFE9FFFE0EBF
:101B3000DBCFEAFFEE52EF04146EFD0EDBCFE9FFC0
:101B4000FE0EDBCFEAFF050EE926000EEA22EF04C7
:101B5000400DF35014100E01436FFD0EDBCFE9FF73
:101B6000FE0EDBCFEAFF020EE926000EEA22EF04AA
:101B7000166EFD0EDBCFE9FFFE0EDBCFEAFF030E94
:101B8000E926000EEA22EF04080DF3CF15F0FD0E52
:101B9000DBCFE9FFFE0EDBCFEAFF070EE926000EE2
:101BA000EA22EF50400DF3CF14F0FD0EDBCFE9FF3A
:101BB000FE0EDBCFEAFF060EE926000EEA22EF500A
:101BC000800DF350141015101610446FFD0EDBCF6E
:101BD000E9FFFE0EDBCFEAFF040EE926000EEA2243
:101BE000EF04156EFD0EDBCFE9FFFE0EDBCFEAFF43
:101BF000090EE926000EEA22EF50400DF3CF14F053
:101C0000FD0EDBCFE9FFFE0EDBCFEAFF080EE92673
:101C1000000EEA22EF50800DF35014101510456F9E
:101C20007D95E66AE668070EE66EE66AE66AF80EF5
:101C3000E66E0E0EE66E90EC18F0146E070EE15E86
:101C400014500E01466B476B4681E66AFD0EDBCFF2
:101C5000E9FFFE0EDBCFEAFFEF50156A000F146EAE
:101C6000010E1522166A176A15AE02D0166817689B
:101C700014C0E6FF15C0E6FF16C0E6FF17C0E6FF7A
:101C8000E00EE66E0E0EE66E90EC18F0186E070E83
:101C9000E15E18500E01FC0E796FF00E716F7269E3
:101CA000200E706EE66A7CEC18F0E552606A0F0157
:101CB000306B0E01806BFD0EDBCFE9FFFE0EDBCF3C
:101CC000EAFFEF50E66ECCEC14F0E552010EE5525F
:101CD000E7CFD9FF1200D9CFE6FFE1CFD9FFE65217
:101CE000FD0EDBCFE9FFFE0EDBCFEAFFEFCFDFFF1C
:101CF000DF50120DF3CFE9FFF4CFEAFF000EE92623
:101D0000010EEA22DFCFEFFFFD0EDBCFE9FFFE0E73
:101D1000DBCFEAFFEE52EECF14F0EECF15F0EECFB0
:101D200016F0EFCF17F0DF50120DF3CFE9FFF4CF2D
:101D3000EAFF000EE926010EEA22EE5214C0EEFF81
:101D400015C0EEFF16C0EEFF17C0EEFFFD0EDBCF95
:101D5000E9FFFE0EDBCFEAFF050EE926000EEA22C0
:101D6000EF50E66EDF50120DF3CFE9FFF4CFEAFF3C
:101D7000000EE926010EEA22050EE926000EEA22EF
:101D8000E552E750EF6EFD0EDBCFE9FFFE0EDBCF35
:101D9000EAFF060EE926000EEA22EECF14F0EECF9F
:101DA00015F0EECF16F0EFCF17F0DF50120DF3CF96
:101DB000E9FFF4CFEAFF000EE926010EEA22060E43
:101DC000E926000EEA2214C0EEFF15C0EEFF16C091
:101DD000EEFF17C0EEFF010EE552E552E7CFD9FF47
:101DE0001200D9CFE6FFE1CFD9FF020EE126DF6A6C
:101DF000010EDB6ADB6A320EF36E010EDBCFF4FFFD
:101E0000F350F45C33E2E66AFD0EDBCFE9FFFE0E31
:101E1000DBCFEAFF050EE926000EEA22EF50E66E60
:101E2000FB0EDBCFE6FFFC0EDBCFE6FFFD0EDBCFCC
:101E3000E9FFFE0EDBCFEAFFEE52EECFE6FFEECF7C
:101E4000E6FFEECFE6FFEFCFE6FFF9EC15F0146EFC
:101E5000080EE15E1450DF6EDF5008E10B0EE66EF7
:101E600007EC21F0E552010EDB2AC5D7DF50146ED6
:101E7000020EE15C02E2E16AE552E16E1450E552C5
:101E8000E7CFD9FF1200D9CFE6FFE1CFD9FF020E8D
:101E9000E126010EDB6AD9CFE6FFDACFE6FFFD0EC1
:101EA000DBCFE9FFFE0EDBCFEAFF050EE926000ED1
:101EB000EA22E9CF14F0EACF15F0E9CFE6FFEACF46
:101EC000E6FFFB0EDBCFE6FFFC0EDBCFE6FFFD0EF1
:101ED000DBCFE9FFFE0EDBCFEAFFEE52E9CF16F0D3
:101EE000EACF17F0E9CFE6FFEACFE6FF4CEC17F0B8
:101EF000186E080EE15E1850E76E010EE7CFDBFFAB
:101F0000080EDF140101CE6F010EDB50146E020EBD
:101F1000E15C02E2E16AE552E16E1450E552E7CF7E
:101F2000D9FF1200D9CFE6FFE1CFD9FF040EE12699
:101F3000DF6A010EDB6A020EDB6A030EDB6ADF6A10
:101F4000DFCF14F0060EE76E1418E8AE02D0E734C7
:101F500002D0E750145C01E3B5D0040EDF02F35069
:101F6000E66E4BEC02F0E552020EF3CFDBFF030E00
:101F7000F4CFDBFF0101D551200DF350E00B01013F
:101F8000C66F020E030EDBCF17F017C016F0176AEC
:101F9000C65100011610E8CFC6F1FF0EE76E020E23
:101FA000DBCF14F0030EE7501416156A14C0C7F106
:101FB000040EDF02F328E66E4BEC02F0E552020E4F
:101FC000F3CFDBFF030EF4CFDBFF020E030EDBCFFC
:101FD00015F015C014F0156A14C0C8F1FF0EE76EB5
:101FE000020EDBCF14F0030EE7501416156A14C06E
:101FF000C9F1040EDF02F350020FE66E4BEC02F063
:10200000E552020EF3CFDBFF030EF4CFDBFF020E2F
:10201000030EDBCF15F015C014F0156A14C0CAF119
:10202000FF0EE76E020EDBCF14F0030EE75014161E
:10203000156A14C0CBF1040EDF02F350030FE66EF5
:102040004BEC02F0E552020EF3CFDBFF030EF4CFB0
:10205000DBFF020E030EDBCF15F015C014F0156A7E
:1020600014C0CCF1FF0EE76E020EDBCF14F0030EAE
:10207000E7501416156A14C0CDF1C60EE66E010EB7
:10208000E66EDF28146E156A14BE1568120E15026E
:10209000F3CF15F01402F3CF14F0F4501526000E10
:1020A0001426010E152214C0E6FF15C0E6FF99DEC6
:1020B000E552E552E552E552E76E010EE7CFDBFF50
:1020C000DF2A3ED7010EDB50146E040EE15C02E203
:1020D000E16AE552E16E1450E552E7CFD9FF1200F4
:1020E000D9CFE6FFE1CFD9FF080EE126060EDB6A65
:1020F000D9CFE6FFDACFE6FFA1EC03F0E552E552D7
:10210000030EDB50E76E070EE7CFDBFFDBCF14F0EB
:10211000000EE76E1418E8AE02D0143403D0E75076
:10212000D88014540DE2070EDBCF15F0460EE76E93
:102130001518E8AE02D0E73402D0E750155C03E38F
:102140000E01010E0E6F0101D651040DF3CF14F0F4
:102150000101D551200DF35014240101C66F070E63
:10216000DBCFC7F1040E0101D603F350E66EA5ECF8
:1021700002F0E552F3CFC8F1040E0101D603F328B3
:10218000E66EA5EC02F0E552F3CFC9F1040E0101B1
:10219000D603F350020FE66EA5EC02F0E552F3CF42
:1021A000CAF1040E0101D603F350030FE66EA5EC4D
:1021B00002F0E552F3CFCBF10101CC6BCD6BC60E33
:1021C000E66E010EE66E900EE66E010EE66E09DE1C
:1021D000E552E552E552E552E76E060EE7CFDBFF2A
:1021E000DB50146E080EE15C02E2E16AE552E16E3A
:1021F0001450E552E7CFD9FF1200D9CFE6FFE1CF67
:10220000D9FF090EE126080EDB6AD9CFE6FFDACF47
:10221000E6FF000EE66E010EE66E35DEE552E55293
:10222000E552E552000919E0010EF36E080EF3CFF6
:10223000DBFF8D70E00EDF14E00BE838E8400101B1
:10224000D86F1F0EDF140101D76FD8C1DAF1010179
:10225000DA2B080EDA5D01E3DA6B080EDB50146E40
:10226000090EE15C02E2E16AE552E16E1450E552CA
:10227000E7CFD9FF1200D9CFE6FFE1CFD9FF090E92
:10228000E126080EDB6AD9CFE6FFDACFE6FF000EC3
:10229000E66E010EE66EF7DDE552E552E552E552D7
:1022A000000976E0010EF36E080EF3CFDBFF7792A4
:1022B0008D70E00EDF14E00BE838E8400101D86FC4
:1022C0001F0EDF140101D76F0101DA510101D85D42
:1022D00003E10101DA2B06D0D8C1DAF10101DA2BD2
:1022E0000101DB2B080E0101DA5D01E3DA6B030E5D
:1022F000DBCFCFF10101D06BD16BD26B080E1F0B7E
:10230000CFC114F0D0C115F0D1C116F0D2C117F071
:1023100007E0D8901436153616361736E806F9E178
:10232000020EDBCF18F0196A1A6A1B6A14501824BF
:102330000101CF6F15501920D06F16501A20D16FA0
:1023400017501B20D26F080E1F0BCFC114F0D0C145
:1023500015F0D1C116F0D2C117F007E0D8901436AD
:10236000153616361736E806F9E1010EDBCF18F000
:10237000196A1A6A1B6A145018240101CF6F15508C
:102380001920D06F16501A20D16F17501B20D26F12
:10239000080EDB50146E090EE15C02E2E16AE552C0
:1023A000E16E1450E552E7CFD9FF1200D9CFE6FF16
:1023B000E1CFD9FF1C0EE126030EF36E080EF3CF1A
:1023C000DBFF090EDB6A0E0EF36E0A0EF3CFDBFFA6
:1023D0000B0EDB6A0C0EDB6A080EF36E0D0EF3CFEC
:1023E000DBFF0E0EDB6A0F0EDB6A100EDB6A110ECE
:1023F000DB6AD950120FE66E000EDA20E66ED95075
:102400000D0FE66E000EDA20E66ED9CFE6FFDACFCA
:10241000E6FFD9500E0FE66E000EDA20E66E4CECA9
:1024200017F0146E080EE15E1450E76E0C0EE7CF45
:10243000DBFF120EDB50080B0101CE6FD9500E0FDF
:10244000E96EDACFEAFFEE5065E1030EEE1862E1C5
:10245000EE5060E1EE505EE1070EDBCFE6FF060EC8
:10246000DBCFE6FF050EDBCFE6FF040EDBCFE6FF9A
:10247000030EDBCFE6FF020EDBCFE6FF010EDB50E3
:10248000DF18E552E718E552E718E552E718E5527C
:10249000E718E552E718E552E718E76E0B0EE7CFAD
:1024A000DBFF080EDB50F36E0B0EDB50F35C0CE130
:1024B0000101400EDD6F0101F36BF3C1E6FF6CDA41
:1024C000E552E66AF50E0CD0090EDB50F36E0B0EEA
:1024D000DB50F35C15E10101800EDD6FE66AF60E5C
:1024E000E66E0D0EE66EE66AE66AF80EE66E0E0E13
:1024F000E66E90EC18F0146E070EE15E14500AD0F0
:102500000A0EDB50F36E0B0EDB50F35C03E10101AE
:102510000A0EDD6F0101DD510A0A01E111D18A0ABB
:1025200001E183D0C00A01E012D1D9500E0FE96E4B
:10253000DACFEAFF0A0EEE1808E1010EEE1805E107
:10254000EE5003E1EE5001E110D9D9500E0FE96EC3
:10255000DACFEAFF0A0EEE1801E0F9D0030EEE180A
:1025600001E0F5D0EE5001E0F2D0EE5001E0EFD006
:10257000130EDB6A0D0EDB50F36E130EDBCFF4FF90
:10258000F350F45C20E2D9CF16F0DACF17F0130E37
:10259000DB500F01D924E96E000EDA20EA6EEF500D
:1025A000E66ED950140F146EDACF15F0130EDB500F
:1025B0001424E96E000EDA20EA6EE552E750EF6E61
:1025C000130EDB2AD7D7140EDB500101F45D01E0B6
:1025D000BED0150EDB50F55D01E0B9D0160EDB5014
:1025E000EB5D01E0B4D0180EDB50EE5D01E0AFD042
:1025F0001B0EDBCFE6FFD0D9E552E66AE6680D0E8A
:10260000E66EE66AE66AF80EE66E0E0EE66E90EC90
:1026100018F0146E070EE15E14501B0EDBCFE6FFC0
:102620000D0EE66EABEC1EF088D0D9500E0FE96EA1
:10263000DACFEAFF090EEE1806E1030EEE1803E109
:10264000EE5001E1EE5002E0000E01D0010E146EDA
:10265000D9500E0FE96EDACFEAFF080EEE1806E148
:10266000030EEE1803E1EE5001E1EE5002E0000E21
:1026700001D0010E14106BE0130EDB6A0D0EDB505F
:10268000F36E130EDBCFF4FFF350F45C20E2D9CFEE
:1026900016F0DACF17F0130EDB500F01D924E96ED4
:1026A000000EDA20EA6EEF50E66ED950140F146E69
:1026B000DACF15F0130EDB501424E96E000EDA2089
:1026C000EA6EE552E750EF6E130EDB2AD7D7D950EA
:1026D0000E0FE96EDACFEAFF080EEE1814E1030ED2
:1026E000EE1811E1EE500FE1EE500DE1D950140F4C
:1026F000E66E000EDA20E66EE66A4FEC1DF0E5525B
:10270000E552E55224D0D9500E0FE96EDACFEAFF38
:10271000090EEE181CE1030EEE1819E1EE5017E158
:10272000EE5015E1D950140FE66E000EDA20E66E79
:10273000080EE66E4FEC1DF0E552E552E55201D071
:1027400014D80101200ED76F0101010EDD6F0C0EB0
:10275000DB50146E1C0EE15C02E2E16AE552E16EB0
:102760001450E552E7CFD9FF1200D9CFE6FFE1CFF1
:10277000D9FF060EE126DF6A010EDB6A020EDB6A74
:10278000030EDB6A040EDB6AF36E050EF3CFDBFF8C
:10279000F4C1C6F1F5C1C7F1EBC1C8F1F6C1C9F189
:1027A000EEC1CAF1F7C1CBF1F1C1CCF1F2C1CDF16B
:1027B0000101F551E66ED950010FE96EDACFEAFF5B
:1027C000E552E750EE6EED6A010EDBCF14F0020E1B
:1027D00014C015F0146A010E14C0DBFF020E15C000
:1027E000DBFFF451E76E010EDBCF14F0020EDBCFFE
:1027F00015F0E7501412010E14C0DBFF020E15C0D5
:10280000DBFF010EDB2A020E01E3DB2A030EDBCF26
:1028100014F0040EDBCF15F0010EDBCF16F0020E24
:10282000DBCF17F01450165C155017580CE3050E4B
:10283000DBCFE6FFD9EC20F0E552030EDB2A040ED5
:10284000E5E3DB2AE3D7C60EE66E010EE66EA20EC6
:10285000E66E010EE66EF1EC0EF0E552E552E55241
:10286000E552DF6EDF50146E060EE15C02E2E16AB3
:10287000E552E16E1450E552E7CFD9FF1200D9CFEF
:10288000E6FFE1CFD9FF070EE126060EDB6A0E0157
:102890000B6B0C6B0D6BD9CFE6FFDACFE6FFF4ECD8
:1028A00002F0E552E552DECF14F0DDCF15F0400E18
:1028B0001416000E1516060ED89015321432E804C0
:1028C000FBE114C00CFE040EDBCF14F0050EDBCFD1
:1028D00015F0010E145C000E155803E30E01010EF5
:1028E0000D6F0101C66B0101D551200DF35001019F
:1028F000D7250101C66FC76B0E010A51400DF3CFFA
:10290000C7F10B51200DF3500101C7130E010C3913
:10291000F00B0101C7130E010D51080DF350010119
:10292000C7130E010E51040DF3500101C7130E0120
:102930000F51E8240101C7130E0110510101C71303
:10294000DFC114F0156ADFC1C8F10101DE510101D8
:10295000C96FCA6BCB6BCC6BCD6BC60EE66E010E2E
:10296000E66E7E0EE66E010EE66EF1EC0EF0E552BE
:10297000E552E552E552E76E060EE7CFDBFFDB508E
:10298000146E070EE15C02E2E16AE552E16E14505A
:10299000E552E7CFD9FF1200D9CFE6FFE1CFD9FF4B
:1029A0000101006BFE0EDB50016F026B000E012770
:1029B000010E0223036B046B02AF02D003690469AA
:1029C000050E056FFE0EDB50066F076B000E062727
:1029D000010E0723086B096B07AF02D0086909696C
:1029E000126FFE0EDB50136F146B000E1327020ED6
:1029F0001423156B166B14AF02D015691669080EF7
:102A0000176F186B196B1A6B1B6B020E246FFE0E7F
:102A1000DB50256F266B010E2527020E2623276B20
:102A2000286B26AF02D027692869080E296F2A6B08
:102A30002B6B2C6B2D6B030E366FFE0EDB50376F3E
:102A4000386B020E37273823396B3A6B38AF02D018
:102A500039693A69080E3B6F3C6B3D6B3E6B3F6BCF
:102A6000040E486FFE0EDB50496F4A6B030E492778
:102A7000020E4A234B6B4C6B4AAF02D04B694C6938
:102A8000080E4D6F4E6B4F6B506B516B050E5A6FAE
:102A9000FE0EDB505B6F5C6B040E5B27020E5C234B
:102AA0005D6B5E6B5CAF02D05D695E69080E5F6F47
:102AB000606B616B626B636B060E6C6FFE0EDB50BE
:102AC0006D6F6E6B050E6D27020E6E236F6B706B54
:102AD0006EAF02D06F697069080E716F726B736BA5
:102AE000746B756B070E7E6FFE0EDB507F6F806B15
:102AF000060E7F27020E8023816B826B80AF02D08F
:102B000081698269080E836F846B856B866B876B26
:102B1000906FFE0EDB50916F926B070E9127020EA5
:102B20009223936B946B92AF02D093699469080ED1
:102B3000956F966B976B986B996BA26FFE0EDB503F
:102B4000A36FA46B0A0EA327020EA423A56BA66B8A
:102B5000A4AF02D0A569A669080EA76FA86BA96BE0
:0E2B6000AA6BAB6B010EE552E7CFD9FF120056
:022B6E00800ED7
:102B7000E66EC2DAE5520E01010E436FF80E446FA5
:102B8000440E456F200E706E729E728C606A0F014B
:102B9000306B0E01806B906BA06BB06BC06BD06B19
:102BA000F80E7D6F880EE06F220EE16FE46F080E65
:102BB000E56F140EE86F050EE96F070E466F476B61
:102BC000716B110E726F736F746B756B766B776BC5
:102BD000786B500E796F050E7A6F7B6B7B6BF869A3
:102BE000F969F997FC6BFD6BFD97E66A85DAE552AA
:102BF0001200D9CFE6FFE1CFD9FF1A0EE126D95056
:102C0000060FE96EDACFEAFF200EEE6E0F0EED6EC4
:102C1000D950080FE96EDACFEAFF100EEE6E0F0EF4
:102C2000ED6ED9500A0FE96EDACFEAFF000EEE6EB4
:102C30000F0EED6ED9500C0FE96EDACFEAFF800E61
:102C4000EE6E0E0EED6ED9500E0FE96EDACFEAFF82
:102C5000900EEE6E0E0EED6ED950100FE96EDACFBB
:102C6000EAFFA00EEE6E0E0EED6ED950120FE96E59
:102C7000DACFEAFFB00EEE6E0E0EED6ED950140FE5
:102C8000E96EDACFEAFFC00EEE6E0E0EED6ED95091
:102C9000160FE96EDACFEAFFD00EEE6E0E0EED6E75
:102CA0000E017D417F0BE76E190EE7CFDBFFDF6A78
:102CB000DF50146E156A080E145C000E155801E3FF
:102CC000DED0D950060F146EDF50020D1450F324DD
:102CD000E96EDA50F420EA6E020EEECFDBFF030E4F
:102CE000EDCFDBFF020EDBCF08F0030EDBCF09F0E8
:102CF000040E08C0DBFF050E09C0DBFFDF50020831
:102D000010E2190EDBCFF3FFF390F342F3CFDBFFBA
:102D1000D950190FE96EDACFEAFFEF50010B01E14C
:102D2000ACD0020EDBCFE9FF030EDBCFEAFFEF50A2
:102D3000080B01E0A2D0FC0E146E020EDBCFE9FFFF
:102D4000030EDBCFEAFF1450EF16F70EDB50030B38
:102D5000146E020EDBCFE9FF030EDBCFEAFF145047
:102D6000EF12F70EDBAC04D0F80EDB50400902D0B6
:102D7000F80EDB50E76E180EE7CFDBFF050EE76EAF
:102D8000020EDBCFE9FF030EDBCFEAFFE750E926B7
:102D9000000EEA22180EDBCFEFFFF70EDBAA06D0FB
:102DA000010EF36E180EF3CFDBFF02D0180EDB6AB4
:102DB000DBCFE6FFD950FB0FE96EFF0EDA20EA6E9B
:102DC000EECFE6FFEECFE6FFEECFE6FFEFCFE6FF7A
:102DD000010EE76E020EDBCF14F0030EDBCF15F011
:102DE000E7501426000E152214C0E6FF15C0E6FFBA
:102DF00097D9166E070EE15E1650D950020FE96E94
:102E0000DACFEAFF060EEE26000EED22010EDB6A97
:102E1000F80EDB50F36E010EDBCFF4FFF350F45CE1
:102E20001AE2F90EDBCFE9FFDB2AFA0EDBCFEAFF6D
:102E300001E3DB2AEF50E66E020EDBCFE9FFDB2A6F
:102E4000030EDBCFEAFF01E3DB2AE552E750EF6E2A
:102E5000010EDB2ADDD7040EDBCFE9FF050EDBCF49
:102E6000EAFFEF50040B07E1040EDBCFE9FF050E8C
:102E7000DBCFEAFFEF86010E03D0DF2A19D7000E61
:102E8000146E1A0EE15C02E2E16AE552E16E145042
:102E9000E552E7CFD9FF1200D9CFE6FFE1CFD9FF46
:102EA000060EE1260E01116B60AE04D0600EDE6EE0
:102EB0000F0E43D00F0130AF04D0300EDE6E0F0E78
:102EC0003CD00E017D51040B07E18051800B04E0E2
:102ED000800EDE6E0E0E31D07D51080B07E1905151
:102EE000800B04E0900EDE6E0E0E27D07D51100B8D
:102EF00007E1A051800B04E0A00EDE6E0E0E1DD087
:102F00007D51200B07E1B051800B04E0B00EDE6E66
:102F10000E0E13D07D51400B07E1C051800B04E031
:102F2000C00EDE6E0E0E09D07D51800B13E1D05124
:102F3000800B10E0D00EDE6E0E0EDD6EDECFE9FFF0
:102F4000DDCFEAFFEF501F0B0E01116F779271ACCE
:102F50000BD002D0000EC4D0F70EDBCFE9FFF80E85
:102F6000DBCFEAFFEF86719CD9CFE9FFDACFEAFF2A
:102F7000020EEECFDBFF030EEDCFDBFFF70EDBCF54
:102F8000E9FFF80EDBCFEAFFEF6ADECFE9FFDDCF26
:102F9000EAFF050EE926000EEA22050EEFCFDBFF61
:102FA000DB500F0BE66EF90EDBCFE9FFFA0EDBCF3D
:102FB000EAFFE552E750EF6ED950050FE96EDACF20
:102FC000EAFFEF50400B07E0F70EDBCFE9FFF80E0A
:102FD000DBCFEAFFEF8CDECFE9FFDDCFEAFF020EA9
:102FE000E926000EEA22050EEFCFDBFFD950050FD0
:102FF000E96EDACFEAFFEF50080B0DE0F70EDBCFFA
:10300000E9FFF80EDBCFEAFFEF8A010EF36E050E43
:10301000F3CFDBFF02D0050EDB6ADBCFE6FFFD0E50
:10302000DBCFE6FFFE0EDBCFE6FFDECF14F0DDCF19
:1030300015F0010E1426000E152214C0E6FF15C06F
:10304000E6FF46D9166E050EE15E1650060EDE2628
:10305000000EDD22F90EDBCFE9FFFA0EDBCFEAFF2F
:10306000050EEFCFDBFF040EDB6ADBCF14F0156A31
:1030700014BE1568050EDB50000115AE02D0D890C5
:1030800003D0145C000E155819E2DFCFE9FFDF2AE8
:10309000010EDBCFEAFF01E3DB2AEF50E66EFB0E09
:1030A000DBCFE9FFDB2AFC0EDBCFEAFF01E3DB2A03
:1030B000E552E750EF6E040EDB2AD7D777AE08D083
:1030C000F70EDBCFE9FFF80EDBCFEAFFEF88779E44
:1030D000020EDBCFE9FF030EDBCFEAFFEF9E010E0E
:1030E000146E060EE15C02E2E16AE552E16E1450F4
:1030F000E552E7CFD9FF1200D9CFE6FFE1CFD9FFE4
:103100001F0E6F16FE0EDB506F12E00E6F14146E62
:10311000FE0EDB50145CF9E1E552E7CFD9FF120057
:10312000D9CFE6FFE1CFD9FF020EE126D950F90F42
:10313000146EFF0EDA2014C0DEFFDD6EF80EDB50D9
:10314000146E156AE850151031E1DECFE9FFDDCFCE
:10315000EAFFEF50E840E840E8401F0BE66EFD0E46
:10316000DBCFE9FFFE0EDBCFEAFFE552E750EF6E63
:10317000DECFE9FFDDCFEAFFEE52EF50200DF3CFB7
:1031800014F0FD0EDBCFE9FFFE0EDBCFEAFFF350BC
:10319000EF12FD0EDB2AFE0E01E3DB2ADECFE9FF94
:1031A000DDCFEAFFEF50200DF3507ED0DECFE9FFF8
:1031B000DDCFEAFF020EE926000EEA22EF50E00B17
:1031C000E838E840E66EFD0EDBCFE9FFFE0EDBCF10
:1031D000EAFFE552E750EF6EDECFE9FFDDCFEAFF11
:1031E000030EE926000EEA22EF50080DF3CF14F08B
:1031F000FD0EDBCFE9FFFE0EDBCFEAFFF350EF124F
:10320000FD0EDB2AFE0E01E3DB2ADECFE9FFDDCF78
:10321000EAFF020EE926000EEA22EF50080DF350F5
:10322000E00BE66EFD0EDBCFE9FFFE0EDBCFEAFF23
:10323000E552E750EF6EFD0EDBCFE9FFFE0EDBCF70
:10324000EAFFEF86DECFE9FFDDCFEAFF020EE926D7
:10325000000EEA22EF50030B146EFD0EDBCFE9FFE8
:10326000FE0EDBCFEAFF1450EF12FD0EDB2AFE0E3E
:1032700001E3DB2ADECFE9FFDDCFEAFFEE52EF50BC
:10328000E66EFD0EDBCFE9FFFE0EDBCFEAFFE55277
:10329000E750EF6EFD0EDB2AFE0E01E3DB2ADECFE8
:1032A000E9FFDDCFEAFFEF50E66EFD0EDBCFE9FF71
:1032B000FE0EDBCFEAFFE552E750EF6E020EE15C57
:1032C00002E2E16AE552E16EE552E7CFD9FF120072
:1032D000D9CFE6FFE1CFD9FF020EE126FB0EDBCF0F
:1032E000DEFFDBCFDDFFFA0EDB50156AE85015106C
:1032F0004CE1FD0EDBCFE9FFFE0EDBCFEAFFEF5026
:10330000080DF350E66EDECFE9FFDDCFEAFFE552B0
:10331000E750EF6EFD0EDBCFE9FFFE0EDBCFEAFFDD
:10332000EF50E00BE838E840E66EDECFE9FFDDCF96
:10333000EAFFEE52E552E750EF6EFD0EDB2AFE0E7D
:1033400001E3DB2AFD0EDBCFE9FFFE0EDBCFEAFF58
:10335000EF50E00BE838E840DECFE9FFDDCFEAFFD1
:10336000E850EF12DECFE9FFDDCFEAFF020EE926DB
:10337000000EEA22EF6ADECFE9FFDDCFEAFF030E9F
:10338000E926000EEA22EF6A84D0FD0EDBCFE9FFCA
:10339000FE0EDBCFEAFFEF50200DF350E66EDECFDE
:1033A000E9FFDDCFEAFF020EE926000EEA22E55230
:1033B000E750EF6EFD0EDBCFE9FFFE0EDBCFEAFF3D
:1033C000EF50E840E840E8401F0BE66EDECFE9FF33
:1033D000DDCFEAFF030EE926000EEA22E552E750B0
:1033E000EF6EFD0EDB2AFE0E01E3DB2AFD0EDBCFC6
:1033F000E9FFFE0EDBCFEAFFEF50030B146EDECFCA
:10340000E9FFDDCFEAFF020EE926000EEA221450A2
:10341000EF12FD0EDBCFE9FFFE0EDBCFEAFFEF5030
:10342000E00BE840E840E8401F0B146EDECFE9FFF8
:10343000DDCFEAFF020EE926000EEA221450EF1259
:10344000FD0EDB2AFE0E01E3DB2AFD0EDBCFE9FFDA
:10345000FE0EDBCFEAFFEF50E66EDECFE9FFDDCFF9
:10346000EAFFEE52E552E750EF6EFD0EDB2AFE0E4C
:1034700001E3DB2AFD0EDBCFE9FFFE0EDBCFEAFF27
:10348000EF50E66EDECFE9FFDDCFEAFFE552E75011
:10349000EF6E020EE15C02E2E16AE552E16EE55296
:0634A000E7CFD9FF120086
:0A34A600DACFE4FFE2CFDAFFE9CF4E
:1034B000E4FFEACFE4FFF6CFE4FFF7CFE4FFF5CF78
:1034C000E4FFF3CFE4FFF4CFE4FFFACFE4FF00EE34
:1034D00000F0140EE80403E3EECFE4FFFBD700EEA8
:1034E00014F00E0EE80403E3EECFE4FFFBD7E65240
:1034F0009D50010B01E1B8D09E50010B01E1B4D009
:10350000B20ECF6ECE6A9E90E2C122F0E3C123F0EC
:10351000E4C124F0E5C125F0030E0B6E0C6A0D6AC0
:103520000E6AE2C106F0E3C107F0E4C108F0E5C1AC
:1035300009F00CEC1FF0025003100410051002E11A
:103540000101D381E2C122F0E3C123F0E4C124F000
:10355000E5C125F00A0E0B6E0C6A0D6A0E6AE2C117
:1035600006F0E3C107F0E4C108F0E5C109F00CEC96
:103570001FF0025003100410051009E10101D3836C
:103580008D72040ED75D03E1E02B000EE123050EE2
:103590000101E21907E1E35105E1E45103E1E551DD
:1035A00001E1D385080EE21907E1E35105E1E45199
:1035B00003E1E55101E1D3850B0EE21907E1E35187
:1035C00005E1E45103E1E55101E1D3850E0EE21975
:1035D00007E1E35105E1E45103E1E55101E1D38560
:1035E000110EE21907E1E35105E1E45103E1E55170
:1035F00001E1D385140EE21907E1E35105E1E4513D
:1036000003E1E55101E1D385E2C122F0E3C123F0FA
:10361000E4C124F0E5C125F0640E0B6E0C6A0D6A5E
:103620000E6AE2C106F0E3C107F0E4C108F0E5C1AB
:1036300009F00CEC1FF002C022F003C023F004C01C
:1036400024F005C025F0025003100410051006E117
:103650000101D387E26BE36BE46BE56B0101E22BC5
:10366000000EE323E423E5237750020B1CE07650A1
:10367000020B19E00101100EDC6F779292EC0FF053
:1036800070EC10F03FEC14F03BEC11F00101E06B3A
:10369000E16BD52BD62B080ED55D01E3D56B060E5D
:1036A000D65D01E3D66BE55200EE21F00E0EE80484
:1036B00003E3E5CFEDFFFBD700EE13F0140EE804B3
:1036C00003E3E5CFEDFFFBD7E5CFFAFFE5CFF4FF4E
:1036D000E5CFF3FFE5CFF5FFE5CFF7FFE5CFF6FF49
:1036E000E5CFEAFFE5CFE9FFE5CFDAFF1100D9CF5B
:1036F000E6FFE1CFD9FFE652D050DF6E000EDB943B
:10370000DB9CDB9EDF501B0A0EE0300A0BE0110A47
:1037100008E0020A05E00B0A01E006D0040005D02B
:1037200004D003D002D001D000D03F0ED01222EC42
:1037300000F0FE0EDBCFD7F1E552E552E7CFD9FF1F
:103740001200D9CFE6FFE1CFD9FF040EE126DE6AF1
:10375000DD6A020EDB6A030EDB6A0101D751100A33
:1037600001E12FD1180A01E122D10C0A01E17BD03D
:10377000060A6FE0220A10E0210A01E052D1FDECB6
:1037800010F0040E0101D75D06E1789276827792FF
:103790000E010F0E7E6F46D1E66A1DEC1DF0E5525C
:1037A000E76E020EE7CFDBFF0101020ED76F020EBC
:1037B000DB50AA0803E00101100ED76FD7C1E6FF66
:1037C00096DFE5525DEC0DF0F3CFDEF1F4CFDFF1E3
:1037D000030EDB6A030EDBCF14F00A0EE76E14183B
:1037E000E8AE02D0E73402D0E750145C18E2040ED1
:1037F000E66ED9EC20F0E5525DEC0DF0F3500101DE
:10380000DE27F4500101DF23DEC1DEF1DFC1DFF18D
:103810000101D890DF33DE33030EDB2ADBD7010151
:10382000CA0EDE5D080EDF5902E3000E01D0010E64
:10383000146E0101BE0ED880DE550A0EDF5502E37C
:10384000000E01D0010E141003E00E01010E0A6FEC
:10385000E9D0ECEC03F0F3CFDEFFF4CFDDFF0101A4
:10386000010ED76FDFD00101D351010B1BE0010125
:10387000D3915DEC0DF0F3500101DE27F45001010E
:10388000DF23DEC1DEF1DFC1DFF10101D890DF33DC
:10389000DE330101D351100B03E05AEC0DF002D0DE
:1038A0000101D3890101D351020B02E00101D3933D
:1038B0000101D351040B0BE00101D3950101D35158
:1038C000400B03E05AEC0DF002D00101D38D010151
:1038D000D351080B26E00101D397040E0101DB5DF3
:1038E00003E30101080ED76F0E010A6B0101CA0E36
:1038F000DE5D080EDF5902E3000E01D0010E146EEA
:103900000101BE0ED880DE550A0EDF5502E3000E1F
:1039100001D0010E141003E00E01010E0A6F010127
:10392000DB6B0101D351A00B39E101010A0ED880F4
:10393000E055000EE15507E20101CF6BD06BD16B72
:10394000D26B3BEC02F0100E0101DC5D27E10101BE
:10395000200EDC6FCFC114F0D0C115F0D1C116F02C
:10396000D2C117F0141E151E161E171E14C0E6FF36
:1039700015C0E6FF16C0E6FF17C0E6FFCFC1E6FFA1
:10398000D0C1E6FFD1C1E6FFD2C1E6FF010EE66E6F
:10399000E3EC05F0186E090EE15E1850D30EE66EEA
:1039A000010EE66ECBEC00F0E552E5523BD0FC0E8A
:1039B0008D148D6E0101010EDD6F0101040ED76FB4
:1039C00031D00101DD052AE1030E8D12F29EF29C39
:1039D00076920101040EDD6FE66AE6680D0EE66E72
:1039E000E66AE66AF80EE66E0E0EE66E90EC18F0E9
:1039F000146E070EE15E14500E014681E66AE66A17
:103A0000010EE66EE66AE66AE00EE66E0E0EE66E01
:103A100090EC18F0146E070EE15E1450D6EC11F025
:103A200001D000D00400040EE15C02E2E16AE5523C
:0A3A3000E16EE552E7CFD9FF120066
:063A3A00D9CFE6FFE1CF49
:103A4000D9FF020EE126010EDB6ADE52120EDD6E98
:103A5000FE0EDB50DF6EDF6A010EDB50DF5C10E232
:103A6000DF50746E7F9E7F9C7F800000DF50EA6A8B
:103A7000E60FE96E010EEA2273CFEFFFDF2AECD7E3
:103A80000101E65100D0146E020EE15C02E2E16A2F
:103A9000E552E16E1450E552E7CFD9FF1200D9CFBD
:103AA000E6FFE1CFD9FF090EE126010EDB6A020E27
:103AB000DB6A030EDB6A040EDB6A050EDB6A060EA8
:103AC000DB6A070EDB6A080EDB6AFE0EDB5027E1BD
:103AD000010EDB6A080EF36E010EDBCFF4FFF3502C
:103AE000F45C01E32ED1010EDB50E76EFC0EDBCF60
:103AF000E9FFFD0EDBCFEAFFE750E926000EEA22E0
:103B0000EF50E66E010EDB28EA6AE60FE96E010E61
:103B1000EA22E552E750EF6E010EDB2ADBD7FE0EFC
:103B2000DB50080801E00DD1010EDB6A040EF36ED4
:103B3000010EDBCFF4FFF350F45C1DE2010EDB500D
:103B4000E76EFC0EDBCFE9FFFD0EDBCFEAFFE750AF
:103B5000E926000EEA22EF50E66E010EDB50090F57
:103B6000EA6AE60FE96E010EEA22E552E750EF6ECF
:103B7000010EDB2ADBD70101AA0EE66FF36B300ED4
:103B8000E75D1A6E1B6A300EE85D1C6E1D6A0A0E38
:103B9000086E096A1CC00DF01DC00EF040EC1FF04D
:103BA0001A500624186E1B500720196E300E0101A2
:103BB000E95D1E6E1F6A640E086E096A1EC00DF074
:103BC0001FC00EF040EC1FF018500624166E19505E
:103BD0000720176E300E0101EA5D206E216AE80EA3
:103BE000086E030E096E20C00DF021C00EF040ECEF
:103BF0001FF016500624146E17500720156EFF0E86
:103C00001416000E1516030E14C0DBFF040E15C0AB
:103C1000DBFF300E0101E75D1A6E1B6A300EE85DB6
:103C20001C6E1D6A0A0E086E096A1CC00DF01DC0CC
:103C30000EF040EC1FF01A500624186E1B5007209F
:103C4000196E300E0101E95D1E6E1F6A640E086E6A
:103C5000096A1EC00DF01FC00EF040EC1FF0185096
:103C60000624166E19500720176E300E0101EA5D0A
:103C7000206E216AE80E086E030E096E20C00DF05A
:103C800021C00EF040EC1FF01650062417500720FC
:103C9000146E156A050E14C0DBFF060E15C0DBFF9F
:103CA000300E0101ED5D0A0D300EEC5DF324E76E80
:103CB000070EE7CFDBFF300EF05D0A0D300EEF5D33
:103CC000F324E76E080EE7CFDBFF030EDBCFF4F142
:103CD000050EDBCFF5F1070EDBCFF6F1080EDBCFDB
:103CE000F7F1120EF36E020EF3CFDBFF010EDB6A6B
:103CF000020EDB50F36E010EDBCFF4FFF350F45CE9
:103D000020E2010EDB50746E010EDB50EA6AE60F12
:103D1000E96E010EEA22EF50736E7F9E7F9C7F84D6
:103D2000F250DF6EF26A550E7E6EAA0E7E6E7F82B4
:103D3000DF50F26E7F94B7ACFED7B79C010EDB2A42
:103D4000D7D7090EE15C02E2E16AE552E16EE55285
:103D5000E7CFD9FF1200D9CFE6FFE1CFD9FFE65276
:103D6000FE0EDB50746EFD0EDB50736E7F9E7F9CEB
:103D70007F84F250DF6EF26A550E7E6EAA0E7E6E62
:103D80007F82DF50F26E7F94B7ACFED7B79CE552CE
:083D9000E552E7CFD9FF120054
:083D9800006A0EAED2EF1EF02E
:103DA0000E6C001E09AED7EF1EF0096C001E15EC5C
:103DB00021F009BEE1EF1EF000AE000C096C056CAD
:103DC000000C00BEDEEF1EF00188FF0C006A0EAE94
:103DD000EFEF1EF00D6C0E1EE86A0E22001E09AEFB
:103DE000F7EF1EF0086C091EE86A0922001EC3ECFA
:103DF00020F009BE07EF1FF000AE000C086C091E92
:103E0000E86A0922046C051EE86A0522000C00BE5F
:103E1000FEEF1EF00188FF0C006AE86A0EAE19EF93
:103E20001FF00B6C0C1E0D1E0E1E0C220D220E22FE
:103E3000001E09AE24EF1FF0066C071E081E091EA7
:103E4000072208220922001E88EC20F009BE3BEF61
:103E50001FF000AE000C066C071E081E091EE86A63
:103E6000072208220922026C031E041E051E0322DB
:103E700004220522000C00BE2BEF1FF00188FF0C6E
:103E800008C012F008500D02F4CF07F0F3CF06F08F
:103E900009500E02F4CF09F0F3CF08F00D02F350F1
:103EA0000726F4500822E86A092212500E02F35045
:0C3EB0000726F4500822E86A0922000CE2
:043EBC009F119711AA
:103EC000901188117F1176116D11641159114F11E4
:103ED000441138112C111F1112110411F610E710A2
:103EE000D710C710B610A51092107F106C10571085
:103EF00042102C101610FF0FE70FCE0FB40F990FC2
:103F00007D0F610F440F260F070FE80EC80EA70E96
:103F1000850E620E3F0E1B0EF60DD10DAB0D850DFD
:103F20005E0D360D0D0DE40CBB0C910C670C3C0CBA
:103F3000120CE60BBA0B8F0B620B360B090BDD0A6A
:103F4000B00A830A570A2B0AFE09D109A509790983
:103F50004D092109F508CA089E08740849081F0878
:103F6000F507CC07A3077A0753072B070407DE06DC
:103F7000B80693066E064A0626060306E105BF0547
:103F80009E057D055D053E051F050005E204C5048F
:103F9000A9048D04710456043C0423040A04F103AB
:103FA000D903C203AB0394037F03690355034003A2
:103FB0002C0319030603F402E202D002BF02AE0290
:103FC0009E028E027E026F0260025202440236029C
:083FD00029021B020F0203028B
:083FD8001E0EF66E000EF76EDE
:103FE000000EF86E0E010900F550056F0900F5503E
:103FF000066F03E1056701D03DD00900F550006F61
:104000000900F550016F0900F550026F0900090021
:10401000F550E96E0900F550EA6E09000900090043
:10402000F550036F0900F550046F09000900F6CF41
:1040300007FEF7CF08FEF8CF09FE00CEF6FF01CE4F
:10404000F7FF02CEF8FF0E01035302E1045307E02D
:104050000900F550EE6E0307F8E20407F9D707CE22
:10406000F6FF08CEF7FF09CEF8FF0E010507000E98
:06407000065BBFD7120041
:0A407600D9CFE6FFE1CFD9FF020E1B
:10408000E126CD0EDF6E010EDB6AFD0EDBCF14F0F4
:10409000FE0EDBCF15F0D890155004E6040E145C2C
:1040A000020E155803E25B0EDF6E25D0010EF76A93
:1040B000DB34FE0BF736F66EBC0EF6263E0EF7220C
:1040C0000900F5CF14F00800F5CF15F0FD0EDBCF99
:1040D00016F0FE0EDBCF17F015501718E8AE02D021
:1040E000173404D01650145C1750155804E3010E11
:1040F000DB2ADF2ADBD7DF50146E020EE15C02E21E
:10410000E16AE552E16E1450E552E7CFD9FF1200A3
:10411000056A046A036A026A200EE76ED8900636C2
:1041200007360836093602360336043605360B5094
:10413000025C0C5003580D5004580E50055809E30A
:104140000B50025E0C50035A0D50045A0E50055A83
:08415000062AE72EE4D7120055
:08415800FF0EE350276EEF0E8D
:1041600001D0F30EE76EE72EB3EF20F00C0E266EB3
:10417000E76AE72EB9EF20F0262EB8EF20F0272EC1
:06418000B1EF20F0120077
:0A418600056A046A100EE76ED89077
:1041900008360936043605360D50045C0E500558B5
:1041A00005E30D50045E0E50055A082AE72EF0D79D
:0241B0001200FB
:0E41B200FF0EE350276E480E01D04C0EE76E54
:1041C000E72EFED7E76AE72EFED7272EF7D70000A7
:0241D0001200DB
:0E41D200410EF36E00EE00F00E0E01D812004A
:1041E000EA6002D0EE6AFCD7F350E9601200EE6A92
:0241F000FCD7FA
:0E41F2001DEE00F02DEE00F0F86A019CECECE2
:0E4200001FF003EC00F0A1EC1BF0FBD7120046
:02420E00FF0EA1
:10421000E350276E1B0E00D001D0200EE76EE72E74
:0A422000FED7272EFAD700D01200B7
:06422A00056A080EE76EB4
:10423000D890093605360E50055C02E3056E092A52
:06424000E72EF7D7120083
:0A424600000000000000000020004E
:0D4250000000002001000000000000000040
:020000040030CA
:0100000015EA
:0100010013EB
:0100030020DC
:00000001FF
